:100000000C941E060C949D280C94CA280C94460649
:100010000C9446060C9446060C9446060C94460630
:100020000C9446060C9446060C941B130C9446063E
:100030000C9446060C9446060C9446060C94460610
:100040000C94F7280C9446060C94E52C0C94282D5F
:100050000C9446060C9446060C9446060C944606F0
:100060000C9446060C944606FC185E193D1940197E
:100070004319461949194C194F195E195819901A04
:10008000921A921A901A921A921A921A921A921A12
:10009000921A921A921A921A921A921A921A921A00
:1000A000161A921A921A921A921A921A8719921A78
:1000B000921A921A921A921A921A921A921A921AE0
:1000C000921A921A921A921A921A921A221A221AB0
:1000D000221A221A221A221A221A221A221A921AD0
:1000E000921A921A921A921A921A8719211A211A9E
:1000F000211A211A921A2F1A351A3B1A411A471A35
:100100004D1A531A591A631A6D1A771A811AC81997
:100110008A19921A921A921A921A161A921A921A04
:10012000921A921A921A921A921A921A201A201A53
:10013000201A201A921A2F1A351A3B1A411A471AF6
:100140004D1A531A591A631A6D1A771A811AC81957
:100150008A19921A921A921A921A161AC51AC51A5E
:10016000C51AC51AC51AC51AC51AC51AC51AC51A97
:10017000C51AC51AC51ADB1BDB1BDB1BDB1BDB1B14
:10018000DB1B0A1B141B1E1B281B851B8F1B9E1BA6
:10019000AF1B371D4C1D581D611D701D951D9E1DEB
:1001A000E71DB01DFA20002106210D211B213D2154
:1001B0005B21456E746572206D656E752E2E2E0066
:1001C000546F67676C6564206D6963726F50504D42
:1001D00000546F67676C656420696E76657274653C
:1001E000642050504D2100546F67676C6564205443
:1001F00058206D7574696E672100546F67676C6570
:10020000642074656C656D65747279210050726F3D
:10021000746F636F6C206572726F72207769746897
:100220002052580054696D656F7574207768656E4B
:1002300020636F6E6E656374696E6720746F205201
:100240005800507265737320616E79206B65792058
:10025000746F2063616E63656C00436F6E6E6563DF
:1002600074696E6720746F2052582C20706F776508
:100270007220757020746865205258202877697440
:10028000682062696E6420706C7567206966206EF4
:100290006F74207573696E6720616C776179732064
:1002A00062696E642900546F67676C656420276912
:1002B0006D6D656469617465206F75747075742700
:1002C00000546F67676C65642027736C61766520E6
:1002D0006D6F64652700546F67676C6564202761E4
:1002E0006C776179732062696E642700546F676769
:1002F0006C65642050504D206368616E6E656C20A3
:100300006C696D69740053657420525353492069B8
:100310006E6A656374696F6E206368616E6E656C8A
:100320002028303D3D64697361626C652900536526
:10033000742050504D206D696E696D756D20737914
:100340006E630053657420626561636F6E20696E31
:1003500074657276616C0053657420626561636FC9
:100360006E2064656C617900536574206265616319
:100370006F6E206672657175656E637920696E2097
:10038000487A3A20303D64697361626C652C205074
:10039000783D504D52206368616E6E656C20782CFC
:1003A0002046783D465253206368616E6E656C202E
:1003B00078005365742050574D2073746F7020641B
:1003C000656C61792028302064697361626C6564B2
:1003D0002C20312D323535203D3D20302E317320FB
:1003E0002D2035306D696E29005365742050504DB5
:1003F0002073746F702064656C61792028302064EC
:10040000697361626C65642C20312D323535203D75
:100410003D20302E3173202D2035306D696E29003E
:10042000536574206661696C736166652064656CF0
:1004300061792028302064697361626C65642C20C6
:10044000312D323535203D3D20302E3173202D2089
:1004500035306D696E29002A2A2A2A2A2A2A2A2A50
:100460002A2A2A2A2A2A2A2A2A2A2A2A2A2A2A2AEC
:100470002A2A2A2A0052582041636B6564202D20C5
:1004800072657665727420737563636573736675E0
:100490006C21002A2A2A2A2A2A2A2A2A2A2A2A2AAD
:1004A0002A2A2A2A2A2A2A2A2A2A2A2A2A2A2A2AAC
:1004B000002A2A2A2A2A2A2A2A2A2A2A2A2A2A2AC6
:1004C0002A2A2A2A2A2A2A2A2A2A2A2A2A2A00528E
:1004D000582041636B6564202D20757064617465DC
:1004E000207375636365737366756C21002A2A2A0D
:1004F0002A2A2A2A2A2A2A2A2A2A2A2A2A2A2A2A5C
:100500002A2A2A2A2A2A2A2A2A2A0056616C696457
:100510002063686F69636573206172653A205B319F
:100520005D2D5B31365D20286368616E6E656C20E1
:10053000312D31362900536574206F7574707574D0
:1005400020666F7220706F727420005B585D2061AE
:10055000626F7274206368616E67657320616E6498
:10056000206578697420525820636F6E6669670051
:100570005B535D20736176652073657474696E6783
:100580007320746F205258005B525D20726576654F
:1005900072742052582073657474696E6773207486
:1005A0006F2064656661756C747300557365206EA9
:1005B000756D62657273205B312D445D20746F2010
:1005C0006564697420706F727473205B452D515D92
:1005D00020666F722073657474696E677300202DD6
:1005E00020726563656976657220636F6E66696700
:1005F000757261746F722C20727820737720000AF4
:100600000A6F70656E4C52536E67200053657420FC
:1006100073657269616C2062617564726174653AB8
:10062000200056616C69642063686F696365733A82
:100630002031202D20342B34202F2032202D203823
:10064000202F2033202D20382B34202F2034202D14
:10065000203132202F2035202D2031322B34202FF5
:100660002036202D20313600536574204368616E9A
:100670006E656C20636F6E6669673A20005365741F
:100680002044617461726174652028302D32293AEA
:10069000200053657420486F70206368616E6E653A
:1006A0006C7320286D61782032342C207365706162
:1006B000726174656420627920636F6D6D61732966
:1006C0002076616C69642076616C75657320312DCC
:1006D0003235353A2000536574206368616E6E656B
:1006E0006C2073706163696E6720287831306B48C5
:1006F0007A293A200053657420524620706F77653E
:10070000722028302D37293A200053657420524634
:10071000206D6167696320286865782920652E67E8
:100720002E20307844454144463030443A2000532E
:1007300065742062617365206672657175656E63AC
:10074000792028696E20487A293A20005B5A5D207A
:10075000656E746572207265636569766572206383
:100760006F6E66696775726174696F6E2075746902
:100770006C79005B465D20646973706C61792061FF
:10078000637475616C206672657175656E63696509
:10079000732075736564005B525D2063616C6375E3
:1007A0006C6174652072616E646F6D206B65792079
:1007B000616E6420686F70206C697374005B495DC2
:1007C000207265696E697469616C697A6520736508
:1007D0007474696E677320746F20736B65746368DB
:1007E0002064656661756C7473005B585D2072658A
:1007F00076657274206368616E67657320616E64EC
:100800002065786974206D656E75005B535D20739B
:100810006176652073657474696E677320746F20E8
:10082000454550524F4D20616E64206578697420B3
:100830006D656E7500557365206E756D62657273BA
:10084000205B302D395D20746F20656469742070E1
:100850006172616D657465727300202D2053797328
:1008600074656D20636F6E66696775726174696F18
:100870006E000A0A6F70656E4C52536E672000510D
:1008800029204F7574707574206265666F726520DB
:100890006C696E6B20283D465329203A2000502970
:1008A00020536C617665206D6F64652028657870D3
:1008B0006572696D656E74616C293A20004F29205C
:1008C00054696D65642042494E44206174207374FC
:1008D000617274757020203A20004E292050504DCE
:1008E000206F7574707574206C696D69746564200F
:1008F000202020203A200044495341424C454400E6
:100900004D292050504D205253534920746F20637D
:1009100068616E6E656C202020203A20004C2920F2
:1009200050504D206D696E696D756D2073796E63E1
:10093000202875732920203A200044495341424C15
:100940004544004B29204661696C736166652062ED
:100950006561636F6E20696E74762E2028312D32AA
:10096000353573293A20004A29204661696C736144
:10097000666520626561636F6E2064656C617920D5
:1009800028302D323535203D3E20313073202D204A
:100990003135306D696E293A200049292046616958
:1009A0006C7361666520626561636F6E206672714B
:1009B0002E203A200048292050574D2073746F7024
:1009C0002064656C6179202020202020203A2000BE
:1009D00047292050504D2073746F702064656C61FE
:1009E00079202020202020203A200046292046611E
:1009F000696C736166652064656C617920202020D4
:100A00002020203A200050574D206368616E6E65AB
:100A10006C200066756E6374696F6E3A2000292041
:100A2000706F72742000506F776572546F776572C3
:100A300000445446205548462033322D62697420C4
:100A400031306368004F70656E4C52536E67525878
:100A5000206D696E6920342F36636800466C7974A6
:100A6000726F6E2F4F72616E6765525820554846FF
:100A70002038636800525820747970653A20004429
:100A8000697361626C656400487A00203D3D200016
:100A900043616C63756C61746564207061636B6540
:100AA0007420696E74657276616C3A200042292068
:100AB0004D6963726F202868616C66292050504D23
:100AC000202020203A00412920496E766572746505
:100AD000642050504D20696E20202020203A0030A4
:100AE00029204D7574652062757A7A657220286DAB
:100AF0006F73746C79293A003929205365726961E2
:100B00006C2062617564726174653A00736D617224
:100B100074506F7274004672536B79005472616E38
:100B200073706172656E740044697361626C6564B0
:100B30000038292054656C656D657472793A2020FF
:100B40002020202020003729204368616E6E656CCC
:100B500020636F6E6669673A202000362920446161
:100B60007461726174652028302D32293A2020206A
:100B700000352920486F70206368616E6E656C7364
:100B80003A2020202020003429204368616E6E65C1
:100B90006C2073706163696E673A202000332920EE
:100BA000524620706F7765722028302D37293A2001
:100BB0002020003229205246206D616769633A2067
:100BC0002020202020202020003129204261736530
:100BD000206672657175656E63793A202020000089
:100BE00000000700020100000304060000000000EE
:100BF00000000001020408102040800102040810D7
:100C00002001020408102004040404040404040263
:100C10000202020202030303030303000000002395
:100C2000002600290000000000250028002B0000FD
:100C3000000000240027002A0000162E11241FBEE9
:100C4000CFEFD8E0DEBFCDBF13E0A0E0B1E0EAE334
:100C5000F2E602C005900D92A83CB107D9F716E064
:100C6000A8ECB3E001C01D92AE38B107E1F71CE07B
:100C7000CCE3DCE004C02297FE010E941F2FCA33A0
:100C8000D107C9F70E94522E0C941B310C9400001E
:100C900080917305813019F482E08093730580910F
:100CA0007305833019F484E0809373050895A89543
:100CB0000895DC01ED91FC910190F081E02D099502
:100CC00008952091740530917505382748E0C901D1
:100CD000880F991F37FF06C09C0151E2252750E17C
:100CE000352701C09C01415091F730937505209341
:100CF0007405089588E38093760580E092ECA1E086
:100D0000B0E08093770590937805A0937905B09330
:100D10007A0587E08093830580E091EAACEBB3E34A
:100D200080937B0590937C05A0937D05B0937E0511
:100D300085E0809384058DEE9EEFADEABEED809355
:100D40007F0590938005A0938105B0938205E5E827
:100D5000F5E080E090E0863028F4DC01AE54BC4F32
:100D60002C9101C020E0219301968831910599F7DB
:100D700082E080939D058AE080939E05089580E03F
:100D80009EECADEEB4E38093BB059093BC05A093BD
:100D9000BD05B093BE0580E090E0A0E0B0E5809393
:100DA000BF059093C005A093C105B093C205E3ECC5
:100DB000F5E080E081938F5F8031E1F70895A0E056
:100DC000B0E0E5EEF6E00C94E82ED82F0E944D2915
:100DD0006115710581059105C9F30E948B2F109251
:100DE0007F05109280051092810510928205C4E063
:100DF000812C912C54018A94C0907F05D09080055D
:100E0000E0908105F0908205FE2CED2CDC2CCC24AA
:100E10000E94862FA50194010E94C72E6C0D7D1D96
:100E20008E1D9F1D60937F057093800580938105C3
:100E300090938205C15001F7DD2309F450C005E805
:100E400015E0E801A12CB12C62E3C62ED12CE12CD7
:100E5000F12C8881882309F442C0B39419F40E94CC
:100E60007A063DC00E94862FA70196010E94C72ED8
:100E7000E1E0E60FA5E8B5E08A2F801B8A1520F493
:100E80008D918E13F9CFE9CF2091840530E0A0E158
:100E9000B7E20E945F2E9B01AC01AE2FB0E00E9432
:100EA0006E2E40907B0550907C0560907D05709083
:100EB0007E05640D751D861D971D4090BB055090E5
:100EC000BC056090BD057090BE05461657066806C5
:100ED000790618F2E993A39488E1A812BACFCDB7A6
:100EE000DEB7E0E10C94042F8436910520F4BC01B8
:100EF00080E090E017C09C018E3B910528F42A55B4
:100F00003109AAE0B0E00CC0823D910528F4245BD1
:100F10003109A4E6B0E004C02D5C3109A8E5B2E0D7
:100F20000E945F2EA4E6B0E09B01AC010E946E2EF1
:100F3000089590E08C599F4F0E947407089582E0B5
:100F40008093B00085E08093B10061E083E00E946F
:100F5000FA2960E083E00E94332A08950097C9F0DF
:100F60009C0140E050E068E478EE81E090E00E946F
:100F7000C72E2F3F31054105510529F020F02FEFF5
:100F800030E040E050E02093B3008091B0008061F9
:100F900003C08091B0008F7E8093B000089560E020
:100FA0008CE00E94FA2961E08BE00E94FA2961E05E
:100FB0008DE00E94FA2960E082E00E94FA2961E057
:100FC00084E00E94FA29089542E050E068E476E067
:100FD00080E00E947D280895E3E0F0E089E08093BE
:100FE0005700E491E67081E0E63009F080E0089572
:100FF000CF93DF93C82F0E94EC07882381F0DFB7DF
:1010000081E080937205F8940E94570688E18093EE
:101010006000C0936000C1110E945706DFBFDF91DE
:10102000CF9108958F929F92AF92BF92CF92DF920D
:10103000EF92FF92CF93FC01C0A5EC2FE770F0E098
:10104000E658FC4FA081B0E0C7FF03C024E130E0C8
:1010500002C02FE030E0FC0197A183E1989FF001EE
:101060001124E25CFE4F80809180A280B380A20FA9
:10107000B31F20E43FE14DE750E00E94792EA50127
:1010800094010E94A52E8C2F887149F469017A0180
:10109000E0EDCE0EE7E0DE1EE11CF11C1BC0C7FF39
:1010A00005C060E47AE88CE29EE004C060E07EEE79
:1010B0008AEB9BE069017A01F8EBCF0EFBE0DF1EC3
:1010C000E11CF11CA50194010E94A52EC20ED31EA5
:1010D000E41EF51EC701B60169517C4F8F4F9F4F2B
:1010E00028EE33E040E050E00E94A52EA8EEB3E0E9
:1010F0000E946E2ECF91FF90EF90DF90CF90BF9027
:10110000AF909F908F9008958F3F910551F048F0D8
:10111000811522E0920738F08115934030F482E087
:10112000089580E0089581E0089583E00895A0E0A7
:10113000B0E0EDE9F8E00C94F12EEB018A01B82F54
:10114000B695A0E028813981F80120832A813B816E
:1011500021832C813D8122832E813F8123836881DD
:1011600079814A815B812C813D81EE81FF819F2FB6
:101170009295990F990F907C272F2370922B252FF2
:101180002370220F220F922B232F23702295207F72
:10119000922BF80194830B5F1F4F2896AF5FBA170D
:1011A00088F680FF24C0888199810E948408D82E07
:1011B0008A819B810E948408E82E8C819D810E94F7
:1011C0008408F82E8E819F810E948408F0E4DF9EBF
:1011D000A001112490E1E99E90011124242B282BD9
:1011E000E4E0FE9EB0011124262BF8012083CDB748
:1011F000DEB7E7E00C940D2F803223E0920708F170
:10120000883E23E0920740F48F519340E4E09695A6
:101210008795EA95E1F70895803D27E0920718F455
:101220008C5D93400895883928E0920768F4885CC3
:10123000974074E0969587957A95E1F78D509C4F8D
:10124000089580E090E008958FEF93E008958C304A
:10125000910540F4A4E0880F991FAA95E1F7885DF5
:101260009C4F0895843F23E0920718F484529C4FCA
:101270000895811524E0920740F48657934FF4E0D7
:10128000880F991FFA95E1F7089580E998E008958D
:101290009C013695279525753575821B930B9C010E
:1012A0002373337396958795969587958373937378
:1012B000820F931F9C0154E0369527955A95E1F7CC
:1012C000280F391F2F703F7041E051E0249FC0016B
:1012D000259F900D349F900D1124892F08952D98EE
:1012E000882319F000002B9A02C000002B98000000
:1012F0002D9A000008952D9A000083B12D980000CA
:10130000829581700895CF93DF93D82F5C9A2D98A2
:101310005C98C8E08D2F80780E946F09DD0FC15066
:10132000C9F72D98DF91CF9108958F770E94830997
:101330000895CF93DF93D82FC8E08D2F80780E9437
:101340006F09DD0FC150C9F72D98DF91CF91089536
:10135000CF93DF932D98C8E080E0D82FDD0F0E9457
:101360007B098D0FC150C9F7DF91CF9108950E947D
:1013700095090E94A8095C9A0895A1E0B0E0E3EC09
:10138000F9E00C94F62E806869830E9483096981D4
:10139000862F0E9499095C9A2196E2E00C94122F04
:1013A000CF93C0917F05C827E82FF0E0EA58FA4FA5
:1013B000678589E70E94BD096C2F8DE30E94BD09F6
:1013C0006C2F82E40E94BD09CF91089586E20E94AD
:1013D000B7090895CF93DF93EC016C818CE10E94F3
:1013E000BD096D818DE10E94BD096E818EE10E9473
:1013F000BD096F8180E20E94BD09688581E20E947B
:10140000BD09698582E20E94BD096A8583E20E9466
:10141000BD096B8584E20E94BD096C8585E20E944E
:10142000BD096D858AE20E94BD096E858EE60E9427
:10143000BD096F858FE60E94BD09688980E70E941B
:10144000BD09698981E70E94BD096A8982E70E9416
:10145000BD09DF91CF910895CF92DF92EF92FF9275
:10146000CF93DF936B017C01C11488E3D8068CE92C
:10147000E8068CE1F80628F5C701B60120E836E950
:1014800048E950E00E94A52EE901689760E879E6F6
:1014900087E69FEF0E94812E6C0D7D1D8E1D9F1D86
:1014A000F2E0660F771F881F991FFA95D1F721E7A1
:1014B00032E040E050E00E94A52EF22EE32E80E4C0
:1014C00021C0C701B60120E03DE241E351E00E94A6
:1014D000A52EE901689760E073ED8EEC9EEF0E9407
:1014E000812E6C0D7D1D8E1D9F1D660F771F881F21
:1014F000991F21E732E040E050E00E94A52EF22E35
:10150000E32E80E66C2F6F71680F85E70E94BD099E
:101510006E2D86E70E94BD096F2D87E70E94BD09E9
:10152000DF91CF91FF90EF90DF90CF900895682FDB
:101530008DE60E94BD0908958F929F92AF92BF924F
:10154000CF92DF92EF92FF92CF93DF93D82F61E09B
:1015500089E00E94332A62E370E080E090E00E941C
:10156000702960E089E00E94332A62E370E080E045
:1015700090E00E94702983E00E94B7098093710572
:1015800084E00E94B7098093700560E086E00E94C5
:10159000BD0961E087E00E94BD096FE789E00E9414
:1015A000BD0965E08AE00E94BD0965E18BE00E940B
:1015B000BD0962E18CE00E94BD096DEF8DE00E94E3
:1015C000BD0960E08EE00E94BD09DD2319F08BE2C9
:1015D00091E008C020919D0533E1239FC0011124B3
:1015E000825C9E4F0E94EA096CE880E30E94BD097C
:1015F0006FE082E30E94BD0962E483E30E94BD09BB
:1016000080919E0587FF02C064E101C06AE084E327
:101610000E94BD096AE285E30E94BD096DE286E38E
:101620000E94BD0964ED87E30E94BD0960E088E384
:101630000E94BD0960E089E30E94BD09D11109C083
:10164000C0907F05D0908005E0908105F0908205E4
:1016500007C0C5E9CC2EC1ECDC2EED2CCEEDFC2E66
:10166000CAE38F2C9924AA24BB24682D8C2F0E94B6
:10167000BD09682D85E08C0F0E94BD09FE2CED2C64
:10168000DC2CCC24CF5FCE3361F76FEF83E40E9474
:10169000BD096FEF84E40E94BD096FEF85E40E94ED
:1016A000BD096FEF86E40E94BD09DD2311F066E0FD
:1016B00002C0609183058DE60E94BD0960E089E764
:1016C0000E94BD09609184058AE70E94BD0960E01F
:1016D00083E70E94BD0960E084E70E94BD09D11143
:1016E00009C060917B0570917C0580917D0590918A
:1016F0007E0504C060E071EA8CEB93E30E942C0A43
:10170000DF91CF91FF90EF90DF90CF90BF90AF909F
:101710009F908F90089561E087E00E94BD0964E288
:101720008EE70E94BD0963E088E00E94BD0960E089
:1017300088E00E94BD0965E087E00E94BD0962E083
:1017400085E00E94BD0983E00E94B709809371057E
:1017500084E00E94B70980937005089583E00E9499
:10176000B7098093710584E00E94B70980937005E2
:1017700061E087E00E94BD096AE070E080E090E0EF
:101780000E9470290E948B0B00000895CF92DF9277
:10179000FF920F931F93CF93DF931F92CDB7DEB7C6
:1017A000082F162F8EE399830E94BD09F02EC02EBC
:1017B0009981D92E8C2D8F19811738F4F6016191FA
:1017C0006F018FE70E94BD09F5CF64E085E00E94BC
:1017D000BD0983E00E94B7098093710584E00E94EF
:1017E000B709809370050E944D2960936C05709332
:1017F0006D0580936E0590936F0569E087E00E9408
:10180000BD0981E0809373050F90DF91CF911F9107
:101810000F91FF90DF90CF9008950F931F930E9438
:10182000C60B80917305813099F40E944D29009177
:101830006C0510916D0520916E0530916F05601B50
:10184000710B820B930B603A76488140910548F307
:1018500080917305813031F46EE971E082EE95E09C
:101860000E94392B1F910F9108950F931F93809120
:101870007305823021F41092730581E020C08091BD
:1018800073058130D9F40E944D2900916C051091A7
:101890006D0520916E0530916F05601B710B820BF9
:1018A000930B613A76488140910540F061E087E012
:1018B0000E94BD091092730582E001C080E01F9173
:1018C0000F910895CF93DF93EC014AE050E06D2F24
:1018D00070E082EE95E00E94072C6EE282EE95E0C9
:1018E0000E940B2BBE0184E0769567958A95E1F7FF
:1018F0006F7077274AE050E082EE95E00E94072C57
:101900006EE282EE95E00E940B2BBE016F7077278E
:101910004AE050E082EE95E00E94072CDF91CF91E3
:101920000895D82FC0E0CD1780F45E9A64E670E089
:1019300080E090E00E9470295E9864E670E080E0AC
:1019400090E00E947029CF5FEECF6CE271E080E002
:1019500090E00E947029E6CF0F931F93CF93DF93FF
:10196000EC01062F15E0115051F0CE010E9402311A
:10197000081741F0602FCE010E940A31F4CF82E0B7
:101980000E94910CDF91CF911F910F910895A0E0DB
:10199000B0E0EDECFCE00C94E82E482E562EC0E0B2
:1019A000D0E0612C712CE12CF12C00E010E0411012
:1019B0000CC06090D40586E4689E3001112459E182
:1019C000E52EF12C0AEB15E01EC091E049120FC084
:1019D0006090D405E6E46E9E30011124FBE16F0EA9
:1019E000711C49E2E42EF12C06E715E00CC082E000
:1019F000481209C028E1622E77247394EE24E39400
:101A0000F12C03ED15E043018C0E9D1E109275051F
:101A1000109274053401A62CA818B12CC3010196AC
:101A20006C01AE14BF04A8F4A00EB11E511006C084
:101A3000C3010E940231F501808305C0F501608178
:101A4000C3010E94AC0CF50180810E946106360141
:101A5000E2CFC301511018C0C3010E940231B82E59
:101A6000C6010E9402312B2D30E0322F2227282B75
:101A700080917405909175058217930779F4C0E001
:101A8000D0E05524539493CF3601609175050E94A0
:101A9000AC0C60917405C6010E94AC0CC05EDE4FB8
:101AA000C13E92E0D90708F482CF852DCDB7DEB7CD
:101AB000E0E10C94042F61E082E00E94C70C0895DD
:101AC00060E082E00E94C70C8091D305853020F051
:101AD0001092D3050E945B0D8091D3058093D405AD
:101AE000089561E080E00E94C70C61E081E00E94FF
:101AF000C70C089560E080E00E94C70C882351F075
:101B000060E081E00E94C70C882321F08091760577
:101B1000883349F00E94BF060E947A0681E00E9445
:101B2000DF060E94710D0895882319F06AEA71E0BA
:101B300002C06EEA71E082EE95E00E94392B0895B2
:101B4000FF920F931F93CF93DF9369EC7BE082EEBC
:101B500095E00E94E52A40917B0550917C056091BB
:101B60007D0570917E052AE030E082EE95E00E94CE
:101B70000E2C63EB7BE082EE95E00E94E52A40911B
:101B80007F0550918005609181057091820520E16B
:101B900030E082EE95E00E940E2C6DE97BE082EE53
:101BA00095E00E94E52A4AE050E06091830582EECC
:101BB00095E00E94362C67E87BE082EE95E00E947B
:101BC000E52A4AE050E06091840582EE95E00E94AB
:101BD000362C61E77BE082EE95E00E94E52AC5E8BD
:101BE000D5E0F12C8E0188818823A9F0FF2031F007
:101BF00061EB71E082EE95E00E94082B21964AE0AD
:101C000050E0F801608182EE95E00E94FF2BF39492
:101C1000F8E1FF12E7CF82EE95E00E94132B6BE50F
:101C20007BE082EE95E00E94E52A4AE050E0609178
:101C30009D0582EE95E00E94362C66E47BE082EE04
:101C400095E00E94E52AE0919E05E770F0E0EE0F36
:101C5000FF1FEE57FC4F6081718182EE95E00E947C
:101C6000392B61E37BE082EE95E00E94E52A8091CA
:101C70009E058871883069F028F4811113C068E2EC
:101C80007BE00CC0803141F0883161F46CE07BE096
:101C900005C06CE17BE002C066E17BE082EE95E08E
:101CA0000E94272B68EF7AE082EE95E00E94E52AF9
:101CB00040917705509178056091790570917A058A
:101CC0002AE030E082EE95E00E940E2C6FED7AE083
:101CD00082EE95E00E94E52A8091BF0580710E9406
:101CE000940D66EC7AE082EE95E00E94E52A809100
:101CF000BF0580740E94940D6DEA7AE082EE95E053
:101D00000E94E52A8091BF0580720E94940D60E9CF
:101D10007AE082EE95E00E94E52A86E795E00E944F
:101D20001208AB01BC012AE030E082EE95E00E948F
:101D3000F02B6BE87AE082EE95E00E94E52A86E7D8
:101D400095E00E9412089B01AC0160E472E48FE010
:101D500090E00E94A52EBA01A9012AE030E082EEAF
:101D600095E00E94F02B68E87AE082EE95E00E9410
:101D7000272BCDB7DEB7E5E00C940F2F8F929F9203
:101D8000AF92BF92CF92DF92EF92FF92811107C084
:101D90006FE77AE082EE95E00E94272B2FC090E05B
:101DA0000E94740724E630E040E050E00E94A52E37
:101DB000CA01B9012AE030E040E050E00E94A52EBF
:101DC00049015A016B017C012AE030E0B501A40110
:101DD00082EE95E00E94F02B6EE282EE95E00E948A
:101DE0000B2B2AE030E0B701A60182EE95E00E94BD
:101DF000F02B63E782EE95E00E944B2BFF90EF9073
:101E0000DF90CF90BF90AF909F908F9008951F93D9
:101E1000CF93DF9365E77AE082EE95E00E94E52AB2
:101E200080919F05813041F46CE57AE082EE95E087
:101E30000E94272B10E050C0823019F465E47AE04C
:101E4000F5CF843019F461E37AE0F0CF853091F773
:101E500066E27AE0EBCFC12FD0E0C930D1050CF4B7
:101E600041C068E3610F82EE95E00E940B2B6EE1AA
:101E70007AE082EE95E00E94E52ABE016F5F7F4F17
:101E80004AE050E082EE95E00E94CF2B63E17AE0D9
:101E900082EE95E00E94E52AC156DA4FE981E032F0
:101EA00018F566E07AE082EE95E00E94E52A8981E5
:101EB000803130F06DE673E082EE95E00E94082BF1
:101EC00069816F7070E06F5F7F4F4AE050E082EE93
:101ED00095E00E94D82B1F5F80914805181708F4E1
:101EE000BACF0FC061E3BECFEF70F0E0EE0FFF1F7F
:101EF000EE56FC4F6081718182EE95E00E94392B95
:101F0000EACF6BEE79E082EE95E00E94E52A8091BF
:101F1000B7050E94BE0E60ED79E082EE95E00E946A
:101F2000E52A8091B8050E94BE0E65EB79E082EE4D
:101F300095E00E94E52A8091B9050E94BE0E6AE9EB
:101F400079E082EE95E00E94E52A4091AF0550913C
:101F5000B0056091B1057091B2054115510561055B
:101F6000710539F12AE030E082EE95E00E940E2CF6
:101F700067E679E082EE95E00E94E52A8091B3055C
:101F80000E949907AB01BC012AE030E082EE95E0A7
:101F90000E940E2C63E479E082EE95E00E94E52A2F
:101FA0004AE050E06091B40582EE95E00E94362C44
:101FB00006C06AE379E082EE95E00E94272B6DE18E
:101FC00079E082EE95E00E94E52A6091B505709176
:101FD000B6054AE050E082EE95E00E94202C60E0D9
:101FE00079E082EE95E00E94E52A6091AE056034CA
:101FF00050F470E06F5F7F4F4AE050E082EE95E072
:102000000E94D82B06C067EF78E082EE95E00E9430
:10201000272B6AED78E082EE95E00E94E52A809118
:10202000AD0580FF03C063EB71E002C067EB71E0B8
:1020300082EE95E00E94392B6DEB78E082EE95E020
:102040000E94E52A8091AD0582700E94940D6EE990
:1020500078E082EE95E00E94E52A8091AD058470DB
:102060000E94940D6FE778E082EE95E00E94E52AE9
:102070008091AD0588700E94940DDF91CF911F91E2
:1020800008950F931F93CF93DF93209145052F3F22
:10209000A9F56FEF75E082EE95E00E94E52A85E8EC
:1020A00093E00E94620C6EED75E082EE95E00E9476
:1020B000E52A80914605909147050E94620C6BEAE3
:1020C00075E082EE95E00E94272B68E875E082EECD
:1020D00095E00E94272B60E775E082EE95E00E9474
:1020E000272B6BE475E082EE95E00E94272B82EEB1
:1020F00095E00E94132B0E94070F68C012160CF087
:1021000065C0332727FD30958091480590E0821700
:1021100093070CF45BC066E375E082EE95E00E94E5
:10212000E52A60914505772767FD70954AE050E004
:1021300082EE95E00E94D82B6BE075E082EE95E090
:102140000E94E52A10E008E2809149051817D0F5B1
:10215000C12FD0E0CC0FDD1FC65BDA4F288130E005
:1021600080914505992787FD909501972817390794
:1021700039F56BEB71E082EE95E00E94082B4AE0A6
:1021800050E0602F82EE95E00E94FF2B6FEB71E034
:1021900082EE95E00E94082BE981EF70F0E0EE0FEF
:1021A000FF1FEE56FC4F6081718182EE95E00E9428
:1021B000082B63EC71E082EE95E00E94082B0F5F24
:1021C0001F5FC2CF82EE95E00E94132BDF91CF916B
:1021D0001F910F910895FF920F931F93CF93DF9359
:1021E000C5E8D5E0F12C8E0188818823D1F165EC1A
:1021F00071E082EE95E00E94082B4AE050E06F2DDE
:1022000082EE95E00E94FF2B62ED71E082EE95E098
:102210000E94082B2196F801208130E0A0E1B7E26E
:102220000E945F2E9B01AC01A0918405B0E00E944A
:102230006E2EAB01BC0180917B0590917C05A09135
:102240007D05B0917E05480F591F6A1F7B1F2AE04C
:1022500030E082EE95E00E940E2CF394F8E1FF123C
:10226000C2CFCDB7DEB7E5E00C940F2F1092DF049C
:1022700085E6E0EEF4E0DF011D928A95E9F7089526
:10228000CF93C82F8F3719F0883009F045C0E091FF
:10229000DF04EE23D9F1E150E093DF04F0E0E052F7
:1022A000FB4F10826DE070E082EE95E00E945906CF
:1022B000C0E08091DF04C81760F4EC2FF0E0E0523A
:1022C000FB4F608170E082EE95E00E945906CF5F7F
:1022D000F0CF60E270E082EE95E00E9459066DE07A
:1022E00070E082EE95E00E945906C0E08091DF0424
:1022F000C81778F5EC2FF0E0E052FB4F608170E0FA
:1023000082EE95E00E945906CF5FF0CF67E082EE43
:1023100095E00E940B2B1DC08B3119F40E943611E1
:102320001AC08D30C1F08A30B1F08091DF0484365C
:1023300068F76C2F70E082EE95E00E945906E091FC
:10234000DF0481E08E0F8093DF04F0E0E052FB4F6A
:10235000C08380E001C081E0CF910895CF93C82F62
:102360000E944D296093C8047093C9048093CA04E5
:102370009093CB04C093DD04CC2329F040E051EED0
:1023800060E070E004C040E855E260E070E082EE9A
:1023900095E00E94952DCF9108959091CC04492FFE
:1023A0004F7050E0BA016F5F7F4F292F30E0E4E0BB
:1023B00035952795EA95E1F76217730759F0FA0109
:1023C000E353FB4F808381E0890F8F70907F892BCF
:1023D0008093CC0408956EE770E082EE95E00E9451
:1023E00059060895A3E1B1E0E8EFF1E10C94E92E7C
:1023F000E5E8F5E0712C8191882321F0739428E1C0
:102400007212F9CF66ED71E082EE95E00E94392BF1
:102410004AE050E0672D82EE95E00E94362C80E085
:102420000E949C0A0E948B0B8E010E5F1F4FC12CD5
:10243000D12C7601C39466246A945C2C0E944129B5
:102440004B015C012091840530E0A0E1B7E20E94DD
:102450005F2E9B01AC01C701B6010E94812E209125
:102460007B0530917C0540917D0550917E05620F82
:10247000731F841F951F2091BB053091BC054091AF
:10248000BD055091BE05261737074807590718F4B0
:10249000F801608225C08C2D0E94D00961E070E0B7
:1024A00080E090E00E947029F80110820E9441298A
:1024B000681979098A099B09643F71408105910572
:1024C00040F40E94E609F8019081981778F780831C
:1024D000EDCF50FE03C05D985E9A02C05D9A5E9893
:1024E0002FEFC21AD20AE20AF20A0F5F1F4F8FEFD4
:1024F000C816D104E104F10409F09FCFCE019395F1
:10250000FC01D82E7FEF68EC2E2F281B271510F02A
:1025100051E056C0DE01129651E02FEF41E03D91AF
:10252000321710F0322F01C0452F5F5F5F3F11F06F
:10253000232FF5CF4193242F30E0A1E0B0E0AC0F82
:10254000BD1FA20FB31F5C93413079F0DE01A20FD3
:10255000B31F5C93423049F0AFEFBFEFAC0FBD1F2C
:10256000A20FB31F6C934E3F78F6A2E0B0E0AC0F21
:10257000BD1FA20FB31F7C934D3F30F6A3E0B0E028
:10258000AC0FBD1FA20FB31F6C93BECF452F242FDE
:1025900030E0FC01E20FF31F6081AFEFB0E0AC0F61
:1025A000BD1FA20FB31F2C91621748F44150DC01EC
:1025B000A40FB11D2C9120836C934111E8CF5F5F74
:1025C000571520F3372D369520E0231770F4DC01E2
:1025D000A20FB11D4C91522F530FFC01E50FF11DBD
:1025E00050815C9340832E5FF0CFF5E8EF2EF5E04D
:1025F000FF2E8C01802F8D19871598F4F801C1905A
:102600008F014AE050E06C2D82EE95E00E94FF2B96
:102610006CE282EE95E00E940B2BF701C1927F01E4
:10262000E9CF82EE95E00E94132B81E0CD5EDE4F74
:10263000EFE00C94052F1F920F920FB60F9211240A
:102640001F932F933F934F935F936F937F938F933A
:102650009F93AF93BF93CF93DF93EF93FF93C0917B
:102660008600D09187008091870490918804209102
:10267000A904211155C09E01281B390B8091BF056B
:102680009091C005A091C105B091C20585FD02C021
:1026900036952795253C49E03407B8F140910A0169
:1026A00050E060E070E02CE1B695A795979587958E
:1026B0002A95D1F70097A105B10521F481E090E0BA
:1026C000A0E0B0E084179507A607B707D8F480917B
:1026D0000A018F3FB9F040E080910A01481780F469
:1026E000842F90E0880F991FFC01E757FB4F208152
:1026F0003181FC01E55FFE4F318320834F5FECCFDA
:102700001092AA0410920A010BC02D3B82E03807F8
:1027100020F080910A018031D8F08FEF80930A0178
:10272000D0938804C0938704FF91EF91DF91CF91FC
:10273000BF91AF919F918F917F916F915F914F91D9
:102740003F912F911F910F900FBE0F901F901895E2
:1027500010910A0181E0810F80930A01C9010E9452
:10276000FC08E12FF0E0EE0FFF1FE757FB4F9183CE
:102770008083D6CF83E0809380008AE980938100B4
:102780008091BF0586FD05C08091810080648093A3
:1027900081008FEF9FEF9093890080938800809154
:1027A0006F00806280936F000895CF93DF930E9443
:1027B000600D8091D405843039F58FE00E94662A3F
:1027C000C1E0D0E0892B11F4C0E0D0E080E10E94AC
:1027D000662A892B19F082E090E002C080E090E048
:1027E0008C2B9D2B8230910539F08330910539F087
:1027F000019739F481E006C01092D40505C082E04B
:1028000001C083E08093D405DF91CF9108956F30AC
:1028100018F086958058089589E0689F802D1124CE
:102820000895A0E0B0E0E7E1F4E10C94F02EC82FA9
:102830000E944D29009138041091390420913A04E6
:1028400030913B046B017C01C01AD10AE20AF30A01
:102850009701860149E8C41643E1D406E104F10476
:1028600010F010923C046093380470933904809304
:102870003A0490933B042091A9048FEF820F823099
:10288000D8F5E0913C04EE2309F44EC1E13011F497
:1028900082E0B8C1E03108F034C181E08E0F80934E
:1028A0003C04F0E0E757FB4FC083803109F0ACC136
:1028B000EBE8F4E0213029F4A181A695A69580816A
:1028C00008C080819181A92FA695A695A695969579
:1028D0008795A03148F4B0E090E0AA0FBB1FA55F38
:1028E000BE4F11969C938E931092AA04329684E068
:1028F000E939F807F9F688C1233009F005C1E091FC
:102900003C04E11104C0CF3009F07EC10DC1E831B3
:1029100048F481E08E0F80933C04F0E0E857FB4FD1
:10292000C08372C1E83109F0ECC0C111EAC040E0D7
:1029300050E0ABE0CA01B3E0880F991FBA95E1F708
:10294000A49F9001A59F300D1124F901E757FB4F7B
:102950006081E1817E2F777075956795FC01EE0FA0
:10296000FF1FE55FFE4F71836083F901E657FB4F60
:10297000B081B695B695B695E181FE2FF295FF0F21
:10298000F07E6F2F6B2BE695E695E6957E2F7770A0
:1029900075956795FC01EE0FFF1FE35FFE4F718396
:1029A0006083F901E557FB4FB081B295B695B695B6
:1029B000B370C181DC2FDD0FDD0F6D2F6B2BC29546
:1029C000C695C695C370E281E170EE0FEE0F7E2FC3
:1029D0007C2B75956795FC01EE0FFF1FE15FFE4FA5
:1029E00071836083F901E357FB4FB081B695E181B4
:1029F000FE2FF795FF27F7956F2F6B2BE6957E2F10
:102A0000777075956795FC01EE0FFF1FEF5EFE4F27
:102A100071836083F901E257FB4FB081B295BF70BB
:102A2000E181FE2FF295F07F6F2F6B2BE295EF7017
:102A30007E2F777075956795FC01EE0FFF1FED5E99
:102A4000FE4F71836083F901E157FB4FB081BB1FDB
:102A5000BB27BB1FC181DC2FDD0F6D2F6B2BCC1F64
:102A6000CC27CC1FE281E370EE0F7E2F7C2B759577
:102A70006795FC01EE0FFF1FEB5EFE4F71836083D5
:102A8000F901EF56FB4FB081B695B695E181FE2F67
:102A9000F295FF0FFF0FF07C6F2F6B2BE695E695FD
:102AA0007E2F777075956795FC01EE0FFF1FE95E2D
:102AB000FE4F71836083F901EE56FB4F2081229512
:102AC000269527703181E32FEE0FEE0FEE0F6E2F5C
:102AD000622B732F72957695777075956795FC01CB
:102AE000EE0FFF1FE75EFE4F718360834F5F5F4F06
:102AF0004230510509F01ECF80919F0483FF109250
:102B0000AA0410923C0480C0243009F07DC060917A
:102B10003C0461110BC0C83AB1F4109275051092D3
:102B2000740588EA0E94610681E06CC0613019F486
:102B3000C093370404C0623031F4C09336048C2F44
:102B40000E9461065AC0E09136042E2F30E0220F19
:102B5000331F462F50E0C9010296841795073CF0B9
:102B6000633268F7FA01EA57FB4FC083E8CF2D5F65
:102B70003F4F8C2F90E0609174057091750542175E
:102B8000530749F4982F8827862797279093750530
:102B90008093740532C06817790769F5809137040E
:102BA000813049F5E13118F080E180933604F090EE
:102BB0003604CAE8D4E000E010E00F15D0F4FE01BE
:102BC0003197808190E0982F88272881822B63E0BD
:102BD000969587956A95E1F70E94FC08F801EE0F3B
:102BE000FF1FE55FFE4F918380830F5F1F4F22968B
:102BF000E4CF1092AA0410923C0480913C048823F4
:102C000019F08F5F80933C04CDB7DEB7E8E00C94F9
:102C10000C2FCF93DF93E82FF0E0E654FA4FE185D5
:102C2000E03150F4F894F0E0EE0FFF1FE55FFE4F47
:102C30008081918178945DC08EE08E0F8B3058F446
:102C4000F0E0E25FF10924E62E9FC0012F9F900D76
:102C500011240C964EC0E03F09F446C038F4E1312F
:102C600081F0E23191F0E03139F409C0ED3FB1F18A
:102C7000EE3FB9F1E13F79F180E092E03AC082E1C4
:102C800001C083E10E948F2A34C08FE00E94662A2F
:102C9000C1E0D0E0892B11F4C0E0D0E080E10E94D7
:102CA000662A892B19F082E090E002C080E090E073
:102CB0008C2B9D2B8230910541F08330910541F0A2
:102CC0000197A9F086EA92E014C08CE090E011C070
:102CD00089E591E00EC086E090E00BC08AEF93E0BA
:102CE00008C08FEF93E005C080E090E002C084EF61
:102CF00093E0DF91CF910895A2E2B0E0E2E8F6E13F
:102D00000C94E62E9E012F5F3F4F80E1D9011D926A
:102D10008A95E9F764E072E082EE95E029A33AA390
:102D20000E94392B0E94AE0B1D8A1E8A1F8A188EA4
:102D3000312C212C00E0812C912C5401412C74E782
:102D4000572E7BE8672E72E3772EE0E5CE2EE3EC7C
:102D5000DE2EE12CF12C84EF91E0A0E0B0E08D8F2D
:102D60009E8FAF8FB8A380E09EECADEEB4E3898F69
:102D70009A8FAB8FBC8F80E094E7ABE8B2E3898B8E
:102D80009A8BAB8BBC8B82EE95E00E944D2C892BED
:102D900009F4E1C082EE95E00E947A2C9C01332771
:102DA0002C32310509F442C0ACF42332310509F06C
:102DB000ABC019821A821B821C821D821E821F8256
:102DC000188619861A861B861C861D861E861F86F7
:102DD000188A60C02434310529F02335310509F4FF
:102DE000B2C092C064E482EE95E00E940B2B2AE010
:102DF00030E040E054E76BE872E382EE95E00E9439
:102E0000992B6CE282EE95E00E940B2B2AE030E0D9
:102E100040E05EEC6DEE74E382EE95E00E94992B4B
:102E20006CE282EE95E00E944B2BADCF0F5F043039
:102E300009F0A9CF29813A814B815C81A8EEB3E0EA
:102E40000E946E2E698B7A8B8B8B9C8B2D813E81A1
:102E50004F8158850E946E2E698F7A8F8B8F9C8F41
:102E600029853A854B855C852D8F3E8F4F8F58A3E2
:102E70002D853E854F8558890E946E2E6B017C0101
:102E800060323EE473078105910530F462E38CE122
:102E90000E94BD0900E077CF603345E774078105E4
:102EA000910510F462E2F3CF60345CE975078105A7
:102EB000910510F466E2EBCF80E5C81683ECD806E6
:102EC000E104F10410F462E1E2CF90E6C9169AEE53
:102ED000D906E104F10410F465E1D9CFA0E7CA16E0
:102EE000A1E1DA06A1E0EA06F10410F461E0CFCF37
:102EF000B0EACB16B6E8DB06B1E0EB06F10410F45D
:102F000063E0C5CF65E0C3CF10ED180F1A3008F0AD
:102F10003ACFE1E0F0E0EC0FFD1F24E0029FE00D6E
:102F2000F11D11242081318142815381AAE0B0E05A
:102F30000E946E2E610F711D811D911D6083718332
:102F40008283938320CF49885A886B887C88812C20
:102F5000912C540118CF81149104A104B10489F477
:102F6000C301B2010E942C0A61E070E080E090E0B1
:102F70000E9470291D8A1E8A1F8A188E312C2224D5
:102F80002A948D8D9E8DAF8DB8A188169906AA06BC
:102F9000BB06D0F40E94E6092D893E894F89588DE1
:102FA000280F311D411D511D2D8B3E8B4F8B588F8E
:102FB000381608F4382E821508F4282E3FEF831AAD
:102FC000930AA30AB30A56C0C301B20128EE33E044
:102FD00040E050E00E94A52EBA01A9012AE030E0AD
:102FE00082EE95E00E94F02B6CE282EE95E00E946A
:102FF0000B2B4AE050E0632D82EE95E00E94FF2B00
:103000006CE282EE95E00E940B2B6D897E898F89A0
:10301000988DA50194010E94A52EBA01A9012AE06C
:1030200030E082EE95E00E94F02B6CE282EE95E0BB
:103030000E940B2B4AE050E0622D82EE95E00E9448
:10304000FF2B6CE282EE95E00E944B2B4C0C5D1C3A
:103050006E1C7F1C898D9A8DAB8DBC8D841595055A
:10306000A605B70520F449885A886B887C88812C8E
:10307000912C540129893A894B895C89283E334037
:103080004105510509F07FCEA296E2E10C94022F92
:10309000ACE1B0E0EEE4F8E10C94F02E0E944D2992
:1030A0006B017C0181E00E949C0A14E703E0198314
:1030B00061E0CE0101960E940D0C009373050E9401
:1030C0008B0B6AEF70E080E090E00E9470298091A5
:1030D0007305833089F482EE95E00E944D2C892B94
:1030E00059F40E944D296C197D098E099F09603899
:1030F000734C894C9140D8F280917305833009F468
:103100004FC08FE70E9495090E94A80989838435E2
:1031100011F083E05CC00E94A809109246058093DC
:1031200047050E94A8092091460530914705280FC0
:10313000311D30934705209346050E94A8098093CE
:1031400048050E94A80980934905813110F7F12CA8
:103150000F2D10E08091490590E0880F991F081706
:10316000190740F40E94A809F801E65BFA4F808332
:10317000F394EECF80E7898361E0CE0101960E944F
:103180000D0C83E0809373050E948B0B62E370E06B
:1031900080E090E00E94702980917305833011F4E3
:1031A00082E015C08FE70E9495090E94A8098983D3
:1031B000803509F0AECF0FE915E00E94A809F801AB
:1031C00081938F01F5E00A3B1F07B9F781E06C9608
:1031D000E8E00C940C2F80914505992787FD909588
:1031E000A92FB92FFC013196EB30F10508F066C02C
:1031F000EC5CFF4F0C941D2F62E778E082EE95E0C7
:103200000E94272B85E893E00E94620C6AE578E033
:1032100082EE95E00E94272B65E378E082EE95E050
:103220000E94272B6BE078E082EE95E00E94272B2E
:103230006AEE77E082EE95E00E94272B6DEB77E057
:1032400082EE95E00E94272B67E977E082EE95E019
:103250000E94272B63E777E082EE95E00E94272B00
:103260006CE477E082EE95E00E94272B82EE95E0F9
:103270000E94132B0E94A00D21C06FE277E01AC0BC
:103280006AE077E017C065EF76E014C066ED76E09F
:1032900011C062E976E00EC06DE776E00BC068E62B
:1032A00076E082EE95E00E94272B62E276E002C093
:1032B0006CE076E082EE95E00E94272B6AE070E0F9
:1032C00080E090E00E94702982EE95E00E944D2CF3
:1032D000892B29F082EE95E00E947A2CF5CF089593
:1032E000ACE1B0E0E6E7F9E10C94F02E90914505F1
:1032F0009F3F09F023C1482F50E0FA013A97EF367B
:10330000F10508F00FC1E15CFF4F0C941D2F61E146
:1033100072E0A0C06DE172E082EE95E00E94392B70
:1033200085E789838BE1EFE9F5E0DE0112960190F4
:103330000D928A95E1F76CE1CE0101960E940D0C89
:103340000E948B0B83E08093730568EC70E080E053
:1033500090E00E94702980917305843009F0E2C0EA
:103360008FE70E9495090E94A8098983853509F095
:10337000D9C06DEE74E082EE95E00E94272B6FECD1
:1033800074E082EE95E00E94272B61EB74E096C01A
:1033900065E372E082EE95E00E94392B89E689832D
:1033A00061E0CE0101960E940D0C0E948B0B83E020
:1033B0008093730568EC70E080E090E00E947029D3
:1033C00080917305843009F0ADC08FE70E949509A4
:1033D0000E94A80989838E010E5F1F4F7E014DE177
:1033E000E40EF11C0E94A809F80181938F01EE15EB
:1033F000FF05C1F78BE1FE013296AFE9B5E0019020
:103400000D928A95E1F78981893409F08BC063E9CF
:1034100074E082EE95E00E94272B65E774E082EE6F
:1034200095E00E94272B67E574E048C06FE472E0E6
:1034300082EE95E00E94392B8EEF8093450572C095
:1034400080528750805390914805981708F066C0C5
:103450006EE572E082EE95E00E94392B63C084E154
:103460008093450560E274E029C085E180934505BD
:1034700069EE73E023C086E18093450562EB73E05B
:103480001DC087E18093450568E673E017C088E1B9
:103490008093450567E573E011C089E18093450598
:1034A00063E473E00BC08AE1809345056EE273E04C
:1034B00005C08BE18093450566E073E082EE95E000
:1034C0000E94272B2FC06CEE72E082EE95E00E94E6
:1034D000272B8091AD0591E01DC066ED72E082EE74
:1034E00095E00E94272B8091AD0592E013C061EC1E
:1034F00072E082EE95E00E94272B8091AD0594E06A
:1035000009C066EA72E082EE95E00E94272B809166
:10351000AD0598E089278093AD058FEF8093450531
:103520000E94411082EE95E00E944D2C892B09F4F7
:103530005AC182EE95E00E947A2CF4CF0E9440118D
:10354000882309F450C18091DF04811104C08FEFFA
:103550008093450540C140E050E060E070E080EEBF
:1035600094E00E94942F40914505042F112707FDF8
:103570001095212F312FF8013197EB31F10508F02B
:103580001AC1E255FF4F0C941D2F552747FD50954A
:103590002091480530E0241735070CF40CC18B014D
:1035A0009C01015011092109310900321105210541
:1035B000310558F0C0904905EBE4F5E0F12CD12C31
:1035C000A8E2EA2E415051090FC0FA01E156FA4F24
:1035D00061506083D8C0DF0111972C9130E024172F
:1035E000350729F0F3943296FC10F5CFCAC00E2DA2
:1035F00010E020E030E0061717072807390741F4EC
:103600002081DA01A156BA4F11962C93DD24D39470
:10361000E394E8CF6F3F71058105910511F008F043
:10362000CAC06093B705AFC06F3F710581059105B2
:1036300011F008F0C0C06093B805A5C06F3F7105D8
:103640008105910511F008F0B6C06093B9059BC0E3
:103650002091E00420622037E9F440E050E060E08F
:1036600070E081EE94E00E94942F9B01AC01DC019C
:10367000CB010197A109B1090897A105B10508F08F
:10368000ADC0A4EDB0E30E946E2E6A5E7C4A8A460D
:10369000954E24C02636E9F440E050E060E070E04A
:1036A00081EE94E00E94942F9B01AC01DC01CB01E0
:1036B0000197A109B1090797A105B10508F08EC0CE
:1036C000A8EAB1E60E946E2E645E7C438E46944E5C
:1036D00005C0611571058105910571F08B019C0193
:1036E00014572B4832430130FAE51F07F2E62F0743
:1036F000F2E03F0708F05FC06093AF057093B0053C
:103700008093B1059093B2053EC06F3F710581056E
:10371000910511F008F04FC06093B30534C08B01E0
:103720009C0101501109210931090F3F11052105A3
:10373000310508F040C06093B40525C08B019C01A1
:10374000045C1940210931090D344DE114072105AC
:10375000310528F47093B6056093B50514C0611562
:1037600071058105910521F48FEF8093AE050BC0A3
:103770006134710581059105F0F461506093AE05E7
:1037800002C0DD20C1F08091DE0481111AC0809159
:103790007F0590918005A0918105B09182050196E9
:1037A000A11DB11D80937F0590938005A093810595
:1037B000B093820506C060E772E082EE95E00E9459
:1037C000392B0E9436118FEF809345056AE082EE17
:1037D00095E00E944B2B0E94411005C061E070E013
:1037E00080E090E07BCF6C96E8E00C940C2F6AE5CB
:1037F00072E082EE95E00E94272B62E472E082EE96
:1038000095E00E94272B82EE95E00E944D2C892B9B
:1038100031F082EE95E00E947A2C0E9470190E948D
:103820004818823029F0833051F46DE072E002C014
:1038300064E272E082EE95E00E94272B08958FEFFC
:10384000809345051092DE040E9441108091450549
:103850008E3F69F082EE95E00E944D2C892BB1F3EA
:1038600082EE95E00E947A2C0E947019EFCF0895A5
:103870000F931F93109145051F3F09F0D2C0893463
:1038800009F457C000F5883309F469C058F480334F
:1038900009F477C008F061C08B3109F440C081326F
:1038A000B1F1B9C0813409F487C030F4893309F427
:1038B00066C0803461F1AFC0823409F48EC08634B2
:1038C00009F448C0A8C0823609F487C078F4883566
:1038D00031F128F48235C1F18335E1F09CC08A359D
:1038E00009F494C0813609F467C095C0823761F14C
:1038F00028F4863679F18936E1F08DC0883779F081
:103900008A3709F483C0833709F085C003C061E1B9
:1039100072E015C00E94710D6EE872E004C00E9452
:103920007A0D68EA72E082EE95E00E94392B8EEF04
:1039300070C00E947A060E94BF0667EC72E082EEB9
:1039400095E00E94392B67C081E00E94DF0660EE9F
:1039500072E0F5CF0E94EB105EC080535AC06AEF50
:1039600071E082EE95E00E94272B90919E0588E001
:10397000890F8871977E892B80939E051AC089E0F4
:1039800048C067EE71E082EE95E00E94272B80919F
:10399000BF059091C005A091C105B091C20520E17D
:1039A00082278093BF059093C005A093C105B09373
:1039B000C205109345052FC061ED71E082EE95E0E0
:1039C0000E94272B8091BF059091C005A091C10551
:1039D000B091C20540E4842710C060EC71E082EE33
:1039E00095E00E94272B8091BF059091C005A09182
:1039F000C105B091C20520E282278093BF05909354
:103A0000C005A093C105B093C20502C00E94F71B78
:103A10008FEF80934505809145058E3F09F0D4C016
:103A2000DDC00E944011882309F4D8C08091DF04D2
:103A3000811104C08FEF80934505C6C040E050E07F
:103A400060E070E080EE94E00E94942F00914505C4
:103A5000112707FD1095212F312FF8013197E930FB
:103A6000F10508F0B4C0E753FF4F0C941D2F8B01F4
:103A70009C01015014472B4832430F3F1945224601
:103A8000324008F0A4C060937B0570937C0580935E
:103A90007D0590937E0577C060937F0570938005C8
:103AA000809381059093820581E08093DE046BC052
:103AB000683071058105910508F089C06093830520
:103AC00062C08B019C0101501109210931090A30A2
:103AD00011052105310508F07AC06093840553C0B3
:103AE00061EB71E080EE94E00E94CE3010E0009730
:103AF00099F00E94A830009779F0183130F4E12F46
:103B0000F0E0EA58FA4F87871F5F61EB71E080E0D1
:103B100090E00E94CE30EBCF1831A8F5E12FF0E015
:103B2000EA58FA4F17861F5FF7CF65307105810598
:103B3000910508F04CC060939D0525C08B019C0148
:103B400001501109210931090630110521053105FE
:103B5000F0F520919E05287F262B20939E0513C00B
:103B60008B019C0101501109210931090115124CE9
:103B70002140310560F56093770570937805809357
:103B8000790590937A058091DE04811113C08091AC
:103B90007F0590918005A0918105B09182050196E5
:103BA000A11DB11D80937F0590938005A093810591
:103BB000B09382050E9436118FEF809345056AE02D
:103BC00082EE95E00E944B2B0E94EB1807C060E745
:103BD00072E082EE95E00E94392BECCF1F910F919D
:103BE00008958FEF809345051092DE040E94EB1834
:103BF000809145058E3F69F082EE95E00E944D2C44
:103C0000892BB1F382EE95E00E947A2C0E94381C39
:103C1000EFCF6AE070E080E090E00E94702982EED1
:103C200095E00E944D2C892B29F082EE95E00E94B0
:103C30007A2CF5CF0895CF93C82F682F82EE95E0A8
:103C40000E94A72C90916A059C2790936A05CF91BA
:103C50000895A1E0B0E0EFE2FEE10C94F62E998326
:103C60000E941B1E9981892F0E941B1E2196E2E053
:103C70000C94122F1F93CF93DF93182FEB01109208
:103C80006A0565EB70E082EE95E00E94590662E6F7
:103C900070E082EE95E00E945906812F0E941B1E63
:103CA000CE010E94291EDF91CF911F91089560914E
:103CB0006A0582EE95E00E94A72C0895A1E2B0E08B
:103CC000E4E6FEE10C94F22E7B018A018C3009F4CB
:103CD00053C108F040C0863009F4BCC018F58330E9
:103CE00009F491C070F4813009F472C0823009F097
:103CF00048C26BE170E082E00E943A1E0FE915E0D5
:103D000078C0843009F487C0853009F03AC26091E8
:103D1000490570E0660F771F85E00E943A1E0AE4AD
:103D200015E086C0893009F4A7C070F4873009F423
:103D30009BC0883009F025C261E070E088E00E94F5
:103D40003A1E8091D40523C28A3009F4CAC08B3050
:103D500009F4F2C016C28A3609F475C1D8F4873660
:103D600009F43AC138F4853609F40EC1863609F4EF
:103D70001FC107C2883609F437C1893609F001C26C
:103D800061E070E089E60E943A1E0E947A060E9475
:103D9000BF06F5C18D3609F4D4C138F48B3609F469
:103DA00091C18C3609F49AC1ECC18E3609F4DCC19C
:103DB000873C09F0E6C161E070E087EC0E943A1EA2
:103DC00081E00E941B1E0E94571E10926B05E3C1EA
:103DD00069E270E081E00E943A1E06E715E0F80112
:103DE00081918F010E941B1EF5E00F391F07B9F763
:103DF000D0C1F80181918F010E941B1EF5E00A3BA2
:103E00001F07B9F7C6C161E070E083E00E943A1E67
:103E10000E944818BCC161E070E084E00E943A1E34
:103E200081E00E941B1E0E94571E0E947C16B3C197
:103E30008091490590E0880F991F98012A543540D8
:103E40002817390708F0A5C1F80181918F010E9458
:103E50001B1EEECF62E070E086E00E943A1E85E80D
:103E600093E00E94291E95C161E070E087E00E9406
:103E70003A1E809148058BC186E6898361E0CE01B8
:103E800001960E940D0C0E948B0B83E080937305BA
:103E900068EC70E080E090E00E94702980917305EA
:103EA0008430D9F48FE70E9495090E94A80989837C
:103EB000863469F460E270E089E00E943A1E10E204
:103EC0000E94A8090E941B1E1150D1F762C161E037
:103ED00070E089E00E943A1E52C161E070E089E022
:103EE00053C169E170E08AE00E943A1E81E080934C
:103EF000BA05209172058091BF059091C005A091EF
:103F0000C105B091C205222311F0806801C08F77EE
:103F10008093BF059093C005A093C105B093C205DF
:103F20000AEB15E0F80181918F010E941B1EF5E05C
:103F3000033D1F07B9F72DC161E270E08BE00E94DD
:103F40003A1E8091AA048F3F39F08091AA0491E033
:103F5000980F9093AA0402C08091AA040E941B1E8D
:103F600010E0812F0E9409160E9427090E94291E35
:103F70001F5F1031B1F70DC161E070E08CE00E946D
:103F80003A1E8091D30503C161E070E085E60E948E
:103F90003A1E89E2E816F10409F0F8C0D801E6E714
:103FA000F5E08D91819385E0EF39F807D1F7E7C00F
:103FB00061E070E086E60E943A1EEBE1EE16F10445
:103FC00009F0E4C0D801EFE9F5E08D91819385E037
:103FD000EA3BF807D1F7D3C061E070E087E60E94C2
:103FE0003A1E0E94710DCBC061E070E088E60E942D
:103FF0003A1E85E789838BE1EFE9F5E0DE01129651
:1040000001900D928A95E1F76CE1CE0101960E9434
:104010000D0C0E948B0B83E08093730560E273E0CC
:1040200080E090E00E94702980917305843009F04F
:10403000ADC08FE70E9495090E94A8098983853544
:1040400009F0A4C09CC061E070E08AE60E943A1EBC
:1040500089E6898361E0CE0101960E940D0C0E94E1
:104060008B0B83E08093730560E273E080E090E067
:104070000E94702980917305843009F087C08FE712
:104080000E9495090E94A80989838E010E5F1F4F27
:104090007E01EDE1EE0EF11C0E94A809F80181936A
:1040A0008F01EE15FF05C1F78BE1FE013296AFE9F6
:1040B000B5E001900D928A95E1F78981893409F084
:1040C00065C05DC061E070E08BE60E943A1EF801B9
:1040D00080818093D4050E947A0D51C061E070E028
:1040E0008CE60E943A1EF0E2EF16F10461F487E6D6
:1040F000898380E2F801DE01129601900D928A9583
:10410000E1F761E203C087E4898361E0CE010196B3
:104110000E940D0C0E948B0B83E0809373056CE46E
:1041200074E080E090E00E947029809173058430F3
:1041300069F58FE70E9495090E94A809873431F537
:104140001EC061E070E08DE60E943A1E89E1E8162B
:10415000F104E1F4D801EAEBF5E08D91819385E07B
:10416000E33DF807D1F70BC061E070E08EE60E94F6
:104170003A1EF80180818093D3050E945B0D81E097
:1041800006C061E070E08AEC0E943A1E80E00E9466
:104190001B1E0E94571EA196E6E00C940E2FA0E075
:1041A000B0E0E5EDF0E20C94F02ECAECD3E014E6BA
:1041B00006E035E0F32E44E0E42E53E0D52E62E035
:1041C000C62E82EE95E00E944D2C892B09F49BC0EF
:1041D00082EE95E00E947A2C282F8093350440913E
:1041E000340450E04730510560F7FA01EE52FF4FBA
:1041F0000C941D2F853B29F781E080933404E1CF97
:10420000823609F07DC0C0923404DBCF8093330442
:1042100080933204D0923404D4CF9C01332730935E
:104220003104209330049091320498279093320403
:10423000E0923404C6CF382F2227409130045091A9
:104240003104242B352B309331042093300490918A
:104250003204982790933204F092340425363105C5
:1042600008F4AFCF61E070E08CEC0E943A1E81E070
:104270000E941B1E0E94571E43C020912E043091A5
:104280002F04F901E653FC4F808390913204982764
:1042900090933204C901019690932F0480932E04C9
:1042A00020913004309131048217930708F489CFAC
:1042B0000093340486CF8091320482130BC0609146
:1042C0002E0470912F044AEC53E0809133040E9435
:1042D0005E1E0DC062E070E08BEC0E943A1E809181
:1042E00033040E941B1E80916A050E941B1EFE0162
:1042F000812F11928A95E9F710922F0410922E04C3
:10430000109234045ECFCDB7DEB7E8E00C940C2FEA
:1043100081E080936B0580916B05882349F082EEE4
:1043200095E00E944D2C892BB1F30E94CF20F3CF52
:104330000895AAE2B0E0EFE9F1E20C94EE2E0E94BB
:1043400041296B017C0181E00E949C0A82EE95E08C
:104350000E944D2C892B29F082EE95E00E947A2C48
:10436000F5CF5E9811E072E6B72EE9E2AE2E03E0DB
:104370000E9441296C197D098E099F09693C7105CC
:1043800081059105D0F11123C1F10E9441296B01F2
:104390007C015D9A80ED97E00E94AE07B982E6E766
:1043A000F5E0DE0112968A2D01900D928A95E1F7D3
:1043B0006AE2CE0101960E940D0C5D9880E090E0CB
:1043C0000E94AE07009373050E948B0B62E370E0BE
:1043D00080E090E00E94702980917305843061F440
:1043E000009373058FE70E9495090E94A80911E0C8
:1043F000823419F410E001C011E08EE00E94662AB8
:10440000892B81F411E00EC05E9A5D9A82EE95E0F0
:104410000E947A2C8D309105A9F05CF40A9791F0F6
:104420005E985D9882EE95E00E944D2C892B61F795
:104430009FCF8332910579F08234910589F70E94EC
:104440008821EECF62EB71E082EE95E00E94272B8F
:104450000E94F11DE5CF0E947C16E2CF8F929F92C1
:10446000AF92BF92CF92DF92EF92FF921F93CF93C2
:10447000DF938EE00E94662A892B09F089C068ECE0
:1044800070E080E090E00E94702980E090E00E945F
:10449000AE070E9441294B015C016B017C0180EC5D
:1044A000C80E82E1D81EE11CF11C0E9441296C1546
:1044B0007D058E059F0530F48EE00E94662A892BCB
:1044C000A1F364C08EE00E94662A892B09F05EC0C9
:1044D00080ED97E00E94AE070E9441296B017C01AC
:1044E000D0E0C1E088E4880E86E2981EA11CB11CD1
:1044F00011E08EE00E94662A892B21F58C149D0420
:10450000AE04BF0430F480ED97E00E94AE07D1E026
:10451000F0CF0E9441296C197D098E099F09693CE1
:1045200071058105910528F30E9441296B017C01E9
:10453000C12719F080ED97E002C080E090E00E9472
:10454000AE07D7CF80E090E00E94AE07DD23B9F040
:104550008091D30590E0019665E070E00E94912E75
:104560008093D3050E945B0D0E94D5130E947A0DA3
:1045700064EF71E080E090E00E94702909C080E063
:104580000E94DF060E94F2110E94710D0E94992183
:10459000DF91CF911F91FF90EF90DF90CF90BF9070
:1045A000AF909F908F900895CF92DF92EF92FF92FD
:1045B00080E00E94F8070E94CF0761E089E00E9436
:1045C000FA2960E089E00E94332A61E086E00E94D7
:1045D000FA2961E085E00E94FA2960E08EE00E94FD
:1045E000FA2960E08FE00E94FA2961E08FE00E94E2
:1045F000332A60E080E10E94FA2961E080E10E94B4
:10460000332A60E088E00E94FA2961E088E00E9495
:10461000332A61E081E10E94FA2960E081E10E9491
:10462000332A0E949F0740E052EC61E070E082EE86
:1046300095E00E94952D0E94D5130E947A0D0E944C
:10464000BA138FEF8093AA040E94E40778940E9423
:1046500041296B017C018091AA048F3F59F40E948B
:1046600041296C197D098E099F09603D77408105BC
:10467000910588F380ED97E00E94AE0761E08EE03F
:104680000E94332A5E9A82EE95E00E944D2C892B7F
:1046900029F082EE95E00E947A2CF5CF6DEF72E062
:1046A00082EE95E00E94082B85E893E00E94620C60
:1046B00064E173E082EE95E00E94082B4AE050E04E
:1046C00064E070E082EE95E00E94D82B62E370E037
:1046D00080E090E00E94702982EE95E00E944D2CCF
:1046E00004970CF182EE95E00E947A2C82349105B9
:1046F000D1F482EE95E00E947A2C8E34910599F4E3
:1047000082EE95E00E947A2C8434910561F482EE69
:1047100095E00E947A2C819731F480E090E00E942D
:10472000AE070E94992140917705509178056091DC
:10473000790570917A05DB01CA010197A109B109D8
:104740000497A105B10568F44093A904433029F406
:1047500040EA56E861E070E004C040E052EC61E0FD
:1047600070E082EE95E00E94952D0E942E225E98C8
:1047700080E090E00E94AE070E94BA131092C50438
:104780008091BF0583FF11C080918B05882351F074
:1047900080919205882331F080919905882311F04A
:1047A00087E001C085E08093C50480E00E949C0AF8
:1047B0008091C6040E94D0090E948B0B10923F0486
:1047C00010923E0410923D04F12C8091D4058F1577
:1047D000B0F062E370E080E090E00E94702980ED2C
:1047E00097E00E94AE0762E370E080E090E00E94F4
:1047F000702980E090E00E94AE07F394E6CF8091AC
:104800009E0584FF08C0982F987181E0983109F0C7
:1048100080E00E94AE118FE00E94F807FF90EF90B9
:10482000DF90CF900895EF92FF920F931F93CF9355
:10483000DF938C016EE770E082EE95E00E945906EE
:10484000E801F12CF0E2EF2E8E0188818D57823045
:1048500048F46DE770E082EE95E00E945906888189
:104860008E2588832196F801608182EE95E00E9472
:10487000A72CF394F9E0FF12E7CF6EE770E082EE29
:1048800095E00E945906CDB7DEB7E6E00C940E2FF6
:10489000A9E0B0E0EEE4F4E20C94F62E9091C704A7
:1048A00091110EC09EEF99838A836B8350E05595DA
:1048B00047954C832D83198618861F821E822EC031
:1048C0004091CC04842F90E0B4E095958795BA95FB
:1048D000E1F7242F2F7030E08217930719F18DEF45
:1048E00089831B82FE01349650E0842F90E0A4E07F
:1048F00095958795AA95E1F7242F2F7030E08217C0
:10490000930749F0DC01A353BB4F8C918193405F27
:104910005F5F563051F74093CC045A83CE01019625
:104920000E9413248091C70490E0019666E070E035
:104930000E94912E8093C7042996E2E00C94122FD6
:10494000A0E0B0E0E6EAF4E20C94EF2E6C016EE732
:1049500070E082EE95E00E9459068601E12CF12C70
:10496000C0E0D0E030E2B32EF801608183E8860F2A
:10497000823078F46DE770E082EE95E00E9459068F
:10498000F80160816B2570E082EE95E00E94590687
:1049900004C082EE95E00E94A72CE114F10459F0C6
:1049A000F80180819E01280F311DC901C92FDD2723
:1049B000C80FD91FDD273FEFE31AF30A89E0E81695
:1049C000F10459F028E0E216F10421F48C2F8095CF
:1049D000F60180870F5F1F4FC7CFCDB7DEB7E9E085
:1049E0000C940B2FA9E0B0E0E8EFF4E20C94F62E63
:1049F000E82F362F8091C70490E0019664E270E0C2
:104A00000E94912E8093C70458E9598350E15A833C
:104A1000813089F048F08230B9F08330D9F48B834B
:104A200081EF8C833D8319C085E08B8381EF8C837C
:104A30002F5F2D8312C08B8381EF8C8384E6489F88
:104A4000A00111245D8309C084E08B8381EF8C83F6
:104A5000ED8303C00E94EB1104C0CE0101960E94B9
:104A6000A0242996E2E00C94122FA2E0B0E0EBE340
:104A7000F5E20C94EB2E182F762E2A8349830E94A0
:104A80004D296B017C018091DD048090C8049090D9
:104A9000C904A090CA04B090CB042A81498188231C
:104AA000C1F0D701C60188199909AA09BB094C01AF
:104AB0005D0191EE89169EE29906A104B10420F1F0
:104AC000241708F4422F202F672D812F0E94F224F3
:104AD00013C0D701C60188199909AA09BB094C015D
:104AE0005D0191E3891695E79906A104B10460F090
:104AF000672D812F0E944824C092C804D092C90417
:104B0000E092CA04F092CB042296EDE00C94072FB9
:104B1000A2E2B0E0EEE8F5E20C94EC2E8CE00E940C
:104B2000B70981110DC06CE173E082EE95E00E943F
:104B3000392B5E9A80E00E949C0A0E948B0B5E9843
:104B400082EE95E00E944D2C892B01F182EE95E0DA
:104B50000E947A2C9091A904992319F00E941114B3
:104B6000EFCF40913E0450E09A012F5F3F4F2F71ED
:104B7000332760913F0470E02617370709F3FA01E5
:104B8000E75BFB4F808320933E04DACF809173056F
:104B9000843009F086C00E944D2961157105810598
:104BA000910549F06093B7047093B8048093B904F9
:104BB0009093BA040CC081E090E0A0E0B0E0809354
:104BC000B7049093B804A093B904B093BA04809149
:104BD000AD049091AE0481609093AE048093AD04D7
:104BE00083E0809373058FE70E94950909E614E03E
:104BF0000E94A809F80181938F01F4E002371F0792
:104C0000B9F72091720480916904982F922796FF3A
:104C10003BC090E4922790937204982F9873983336
:104C2000F1F410E0212F30E080916904877090E06A
:104C3000821793074CF11F5F20919E05812F90E012
:104C4000FC01E759FB4F24FF04C080810E94CD1175
:104C5000E9CF608182EE95E00E94A72CE3CF8F73AD
:104C600099F480916A048093B60480916B048093D8
:104C7000B40480916C048093B30480916F0490E03D
:104C80009093AC048093AB0480913D04813019F47F
:104C900082E080933D0480913D04833011F41092B2
:104CA0003D040E944D296B017C018091AF049091DD
:104CB000B004A091B104B091B2040097A105B10570
:104CC000C9F0A7019601281B390B4A0B5B0BDA01CF
:104CD000C901883B9B40A105B10560F00E94E6092F
:104CE0008093B5041092AF041092B0041092B104F6
:104CF0001092B2048091BB049091BC04A091BD04B9
:104D0000B091BE0446015701881A990AAA0ABB0A43
:104D100086E795E00E94120886169706A806B9064F
:104D200008F4B1C0C092BB04D092BC04E092BD04B0
:104D3000F092BE040E9457068091AA048830A0F029
:104D40008091BF059091C005A091C105B091C205A9
:104D50005CE1B695A795979587955A95D1F7892BDC
:104D60008A2B8B2B09F0B8C18091AA048F5F8093A6
:104D7000AA048091B7049091B804A091B904B091AD
:104D8000BA040097A105B105F1F0C81AD90AEA0AD8
:104D9000FB0A86E795E00E9412086C157D058E05DA
:104DA0009F0508F00FC18091BF0584FD04C080ED10
:104DB00097E00E94AE071092B7041092B8041092C8
:104DC000B9041092BA0490917204907C909372048A
:104DD00050913E0480913F0420913D04581709F4FE
:104DE0000EC1223009F00BC1905890937204E091EB
:104DF0009E05E770F0E0E658FC4F6081693008F0EE
:104E0000E6C0615040E04613E4C080933F0487E36E
:104E1000840F90917204892B809372044093400414
:104E200083E080933D045D9A109183058091C504D1
:104E3000811132C18091BF0582FD3AC1812F0E944C
:104E4000970A8091C6040E94D009E0919E05E77000
:104E5000F0E0E658FC4F608182E794E00E94C60BC8
:104E60008091BF0582FD2DC1E091C604EF5FE09304
:104E7000C604E83109F42DC1F0E0EA58FA4F8785FD
:104E8000882309F426C10E94350C813069F5809190
:104E90009E05887149F18091AD049091AE04880F10
:104EA000991F9093AE048093AD0483E080937305C3
:104EB0000E948B0B0E944D296093AF047093B00445
:104EC0008093B1049093B204672B682B692B61F433
:104ED00081E090E0A0E0B0E08093AF049093B00454
:104EE000A093B104B093B20480919E0584FF1FC0CB
:104EF0008091AD049091AE048E7F0E944809182FD6
:104F00006091AB048091B6040E940714482F612F72
:104F10008091B50449A30E9407140091D405282F5D
:104F200049A16091B3048091B4040E9435255D9835
:104F30008091C3048130C1F018F08230B1F1D9C042
:104F40008EE00E94662A892B09F0D3C081E080930D
:104F5000C3040E9441296093BF047093C0048093EE
:104F6000C1049093C204C5C08EE00E94662A892BBA
:104F700031F50E944129C090BF04D090C004E09058
:104F8000C104F090C2046C197D098E099F09693E25
:104F900073408105910508F4ACC082E08093C3049E
:104FA00080ED97E00E94AE07A4C08EE00E94662AC2
:104FB000892B09F49EC080E090E00E94AE07109219
:104FC000C30497C080E090E00E94AE07FCCE68E08A
:104FD00019CF851709F419CF4F5F242F30E090E0E7
:104FE000F901EE58FB4FDC01A75BBB4F7C9170834E
:104FF000F901E05CFB4F708301968F7104CF243080
:10500000B1F42091400481E494E0A3E7B4E0FC0112
:105010003E2F381B321718F431913D93F9CF87E3B7
:10502000820F90917204892B80937204F9CE809143
:10503000C304823051F49160909372045E9A8E01A1
:105040000F5F1F4FF12CB80110C05E9880913D0496
:10505000811103C081E080933D0480913D04833041
:1050600071F784E080933D04EACF8F2D69A37AA382
:105070000E940916F801819391938F01F39469A11D
:105080007AA1F0E1FF12F1CF80919E0543E754E051
:1050900087700E949708C7CE112309F4CBCE909158
:1050A000C40421E0290F2093C4049813C3CE1DC06B
:1050B0008FE00E94662A892B09F0C0CE5E9A17E025
:1050C000BDCE8FE00E94662A892B09F0CDCE5E9876
:1050D000CBCE1092C604D7CE8091AA04883009F4B2
:1050E0005E9A89E08093AA04CECE1092C404115037
:1050F000A1CEA296ECE00C94082F8230E8F4E82FC1
:10510000F0E0EE0FFF1FEB52FA4F718360838130A6
:1051100041F0809169008C7F842B80936900E89A2C
:10512000089580916900440F551F440F551F837FD8
:10513000842B80936900E99A08951F920F920FB60D
:105140000F9211242F933F934F935F936F937F930D
:105150008F939F93AF93BF93EF93FF938091D50568
:105160009091D605892B29F0E091D505F091D605CF
:105170000995FF91EF91BF91AF919F918F917F9191
:105180006F915F914F913F912F910F900FBE0F90B4
:105190001F9018951F920F920FB60F9211242F9304
:1051A0003F934F935F936F937F938F939F93AF93AF
:1051B000BF93EF93FF938091D7059091D805892BEA
:1051C00029F0E091D705F091D8050995FF91EF916D
:1051D000BF91AF919F918F917F916F915F914F910F
:1051E0003F912F910F900FBE0F901F9018951F9217
:1051F0000F920FB60F9211242F933F938F939F938B
:10520000AF93BF938091DA059091DB05A091DC0507
:10521000B091DD053091D90523E0230F2D3720F41F
:105220000196A11DB11D05C026E8230F0296A11D00
:10523000B11D2093D9058093DA059093DB05A093E7
:10524000DC05B093DD058091DE059091DF05A0912E
:10525000E005B091E1050196A11DB11D8093DE0529
:105260009093DF05A093E005B093E105BF91AF9166
:105270009F918F913F912F910F900FBE0F901F9094
:1052800018952FB7F8946091DA057091DB0580913D
:10529000DC059091DD052FBF08953FB7F89480910C
:1052A000DE059091DF05A091E005B091E10526B5FE
:1052B000A89B05C02F3F19F00196A11DB11D3FBF4E
:1052C0006627782F892F9A2F620F711D811D911DDE
:1052D00042E0660F771F881F991F4A95D1F70895FE
:1052E000CF92DF92EF92FF92CF93DF936B017C011D
:1052F0000E944D29EB01C114D104E104F10479F0BD
:105300000E944D296C1B7D0B683E7340A0F381E029
:10531000C81AD108E108F108C851DC4FECCFDF9181
:10532000CF91FF90EF90DF90CF900895789484B55F
:10533000826084BD84B5816084BD85B5826085BD91
:1053400085B5816085BDEEE6F0E080818160808377
:10535000E1E8F0E01082808182608083808181605A
:105360008083E0E8F0E0808181608083E1EBF0E021
:10537000808184608083E0EBF0E0808181608083C5
:10538000EAE7F0E0808184608083808182608083AE
:105390008081816080838081806880831092C100D9
:1053A0000895833081F028F4813099F08230A1F0A3
:1053B00008958630A9F08730B9F08430D1F4809117
:1053C00080008F7D03C0809180008F778093800064
:1053D000089584B58F7702C084B58F7D84BD08950C
:1053E0008091B0008F7703C08091B0008F7D809353
:1053F000B0000895CF93DF9390E0FC01ED50F44F9F
:105400002491FC01E95FF34F8491882349F190E0F6
:10541000880F991FFC01E15DF34FA591B4918B5D5D
:10542000934FFC01C591D4919FB7611108C0F894C6
:105430008C91209582238C93888182230AC06230CC
:1054400051F4F8948C91322F309583238C9388817A
:10545000822B888304C0F8948C91822B8C939FBFFD
:10546000DF91CF910895A1E0B0E0E9E3FAE20C9476
:10547000F42E282F30E0F901E152F44F8491F90124
:10548000ED50F44F1491F901E95FF34F04910023BB
:10549000C9F0882321F069830E94D1296981E02F16
:1054A000F0E0EE0FFF1FEB5DF34FA591B4919FB7B6
:1054B000F8948C91611103C01095812301C0812B58
:1054C0008C939FBF2196E4E00C94102FCF93DF9331
:1054D000282F30E0F901E152F44F8491F901ED50A9
:1054E000F44FD491F901E95FF34FC491CC2391F0CB
:1054F00081110E94D129EC2FF0E0EE0FFF1FE55E35
:10550000F34FA591B4912C912D2381E090E021F4EB
:1055100080E002C080E090E0DF91CF9108958E306E
:1055200008F08E50877020919D0190E4299F900192
:105530001124822B80937C0080917A008064809378
:105540007A0080917A0086FDFCCF809178002091CE
:10555000790090E0922B0895A0E0B0E0E2EBFAE24F
:105560000C94F02E6C017A01EB01E60EF71E00E0C0
:1055700010E0CE15DF0561F06991D601ED91FC9147
:105580000190F081E02DC6010995080F191FF1CF98
:10559000C801CDB7DEB7E8E00C940C2F611571059A
:1055A00089F0DB010D900020E9F7AD014150510970
:1055B000461B570BDC01ED91FC910280F381E02D3D
:1055C0000995089580E090E00895EF92FF920F937F
:1055D0001F93CF93DF938C01FB01C0E0D0E0649177
:1055E0007F018FEFE81AF80A662361F0D801ED9188
:1055F000FC910190F081E02DC8010995C80FD91FD9
:10560000F701EDCFCE01CDB7DEB7E6E00C940E2F5B
:105610000E94CE2A0895DC01ED91FC910190F08169
:10562000E02D099508950F931F93CF93DF93EC011D
:105630006DE00E940B2B8C016AE0CE010E940B2BC7
:10564000800F911FDF91CF911F910F9108950F93BC
:105650001F93CF93DF93EC010E94E52A8C01CE01CA
:105660000E94132B800F911FDF91CF911F910F91FB
:1056700008950F931F93CF93DF93EC010E94CE2ADE
:105680008C01CE010E94132B800F911FDF91CF91CF
:105690001F910F9108950F931F93CF93DF93EC0108
:1056A0000E940B2B8C01CE010E94132B800F911FA7
:1056B000DF91CF911F910F910895A1E2B0E0E3E651
:1056C000FBE20C94EC2E7C01C42EE52FCB01D22EF4
:1056D00019A221E02D1510F02AE0D22E8E010F5DC7
:1056E0001F4F8D2C912CA12CB12C6C2D7E2FA50140
:1056F00094010E94A52E8C2DD29E80191124015058
:1057000011098A3010F4805D01C0895CF801808342
:10571000211531054105510521F0C22EE32FCA01A3
:10572000E4CFB801C7010E94CE2AA196ECE00C9408
:10573000082FA0E0B0E0EFE9FBE20C94F02EEC01C2
:105740006A017B012115310541F4E881F98101905D
:10575000F081E02D642F09951DC02A303105A9F490
:1057600077FF12C06DE20E940B2B8C014427552756
:10577000BA014C195D096E097F092AE0CE010E9429
:105780005D2B800F911F06C02AE0B701A601CE0154
:105790000E945D2BCDB7DEB7E8E00C940C2F9A0188
:1057A000AB01662757FD6095762F0E94992B0895CF
:1057B0000F931F93CF93DF93EC019A01AB01662700
:1057C00057FD6095762F0E94992B8C01CE010E9487
:1057D000132B800F911FDF91CF911F910F9108958F
:1057E0002115310549F4DC01ED91FC910190F08126
:1057F000E02D642F099508950E945D2B08959A016C
:10580000462F50E060E070E00E94F02B08959A016E
:10581000AB0160E070E00E94F02B08950F931F939E
:10582000CF93DF93EC010E94F02B8C01CE010E94FC
:10583000132B800F911FDF91CF911F910F9108952E
:105840000F931F93CF93DF93EC019A01AB0160E0BC
:1058500070E00E94F02B8C01CE010E94132B800F70
:10586000911FDF91CF911F910F9108950F931F9377
:10587000CF93DF93EC019A01462F50E060E070E097
:105880000E94F02B8C01CE010E94132B800F911FE0
:10589000DF91CF911F910F910895FC0124853585EB
:1058A000F901E05CFF4F80819181F901EE5BFF4FD0
:1058B00020813181821B930B8F7399270895FC01FE
:1058C00084859585FC01E05CFF4F40815181FC019E
:1058D000EE5BFF4F208131814217530741F0019069
:1058E000F081E02DE80FF91F808190E008958FEF9F
:1058F0009FEF0895FC0184859585FC01E05CFF4FD6
:1059000040815181FC01EE5BFF4F208131814217C4
:10591000530779F0A081B181A80FB91F8C91208124
:1059200031812F5F3F4F2F7333273183208390E0E6
:1059300008958FEF9FEF0895FC0181A1882329F03E
:10594000A489B5898C9186FFFBCF11A20895CF93CE
:10595000DF93FC0126853785D901A05CBF4F8D916F
:105960009C91119701968F739927E901CE5BDF4FC8
:105970004881598184179507D9F30D90BC91A02DCA
:10598000A20FB31F6C93A685B785A05CBF4F11967D
:105990009C938E93A689B7892C9181E090E0078C27
:1059A00002C0880F991F0A94E2F7282B2C9381E0FC
:1059B00081A30488F589E02D80818064808381E063
:1059C00090E0DF91CF91089508951F920F920FB646
:1059D0000F9211242F933F934F938F939F93EF93A5
:1059E000FF938091C00082FD1CC04091C600809151
:1059F00088069091890601968F73992720918A06CF
:105A000030918B068217930771F0E0918806F09130
:105A10008906E85BF94F4083909389068093880656
:105A200002C08091C600FF91EF919F918F914F919D
:105A30003F912F910F900FBE0F901F90189582EEFF
:105A400095E00E944D2C892B11F00E94E42C0895C2
:105A50001F920F920FB60F9211242F933F938F93A3
:105A60009F93EF93FF9320914406309145068091D8
:105A70004606909147062817390731F48091C100F6
:105A80008F7D8093C10014C0E0914606F0914706D7
:105A9000EC5FF94F20818091460690914706019670
:105AA0008F73992790934706809346062093C600EC
:105AB000FF91EF919F918F913F912F910F900FBE8A
:105AC0000F901F901895A0E0B0E0E9E6FDE20C947D
:105AD000EC2EFC011382128288EE93E0A0E0B0E08D
:105AE00084839583A683B7838CEB93E09183808333
:105AF0007587648757874687318B208B138B028B82
:105B0000F58AE48AD78AC68AB18EA08E938E828E59
:105B10008F85848F8889858F8989868F8A89878FE9
:105B20008B8980A3ECE00C94082FCF92DF92EF9248
:105B3000FF92CF93DF93EC016A017B01411581EE67
:105B4000580761057105F9F0EC89FD8981E090E065
:105B500008A002C0880F991F0A94E2F7808360E0D2
:105B600079E08DE390E0A70196010E94A52E2150D7
:105B700031094109510956954795379527952115C2
:105B800080E1380798F0EC89FD89108260E874E8BC
:105B90008EE190E0A70196010E94A52E21503109C7
:105BA000410951095695479537952795E889F9890F
:105BB0003083EA89FB89208319A2EE89FF8940811D
:105BC00081E090E09C010C8C02C0220F331F0A94EC
:105BD000E2F7422B4083EE89FF8940819C010D8CC6
:105BE00002C0220F331F0A94E2F7422B4083EE8952
:105BF000FF8940819C010E8C02C0220F331F0A9442
:105C0000E2F7422B4083EE89FF8920810F8C02C08E
:105C1000880F991F0A94E2F7809582238083DF9191
:105C2000CF91FF90EF90DF90CF9008958F929F9249
:105C3000AF92BF92CF92DF92EF92FF920F931F939A
:105C400081E08F9385E08F9387E08F9383E08F933C
:105C500084E08F93E6EC8E2E912CF2ECAF2EB12CDB
:105C6000A1ECCA2ED12CB0ECEB2EF12C04EC10E000
:105C700025EC30E044E056E068E476E082EE95E022
:105C80000E94632D0F900F900F900F900F901F9117
:105C90000F91FF90EF90DF90CF90BF90AF909F90CB
:105CA0008F9008950E9496290E94D422CFE1DDE2D0
:105CB0000E9488252097E1F30E941F2DF9CFA29F13
:105CC000B001B39FC001A39F700D811D1124911DD0
:105CD000B29F700D811D1124911D08950E945F2EA9
:105CE000A59F900DB49F900DA49F800D911D112430
:105CF0000895B7FF0C946E2E0E946E2E821B930B9C
:105D00000895DB018F939F930E946E2EBF91AF91F8
:105D1000A29F800D911DA39F900DB29F900D112405
:105D2000089597FB072E16F4009407D077FD09D04D
:105D30000E94232F07FC05D03EF4909581959F4F3C
:105D40000895709561957F4F0895A1E21A2EAA1BC0
:105D5000BB1BFD010DC0AA1FBB1FEE1FFF1FA2171B
:105D6000B307E407F50720F0A21BB30BE40BF50B18
:105D7000661F771F881F991F1A9469F760957095A1
:105D8000809590959B01AC01BD01CF010895052E32
:105D900097FB1EF400940E94DE2E57FD07D00E9450
:105DA000A52E07FC03D04EF40C94DE2E50954095A2
:105DB000309521953F4F4F4F5F4F089590958095B7
:105DC000709561957F4F8F4F9F4F08952F923F920F
:105DD0004F925F926F927F928F929F92AF92BF92FB
:105DE000CF92DF92EF92FF920F931F93CF93DF93A7
:105DF000CDB7DEB7CA1BDB0B0FB6F894DEBF0FBE04
:105E0000CDBF09942A88398848885F846E847D8450
:105E10008C849B84AA84B984C884DF80EE80FD8052
:105E20000C811B81AA81B981CE0FD11D0FB6F894C8
:105E3000DEBF0FBECDBFED010895EE0FFF1F059031
:105E4000F491E02D0994AA1BBB1B51E107C0AA1FC6
:105E5000BB1FA617B70710F0A61BB70B881F991F0B
:105E60005A95A9F780959095BC01CD0108958F9220
:105E70009F92AF92BF92CF92DF92EF92FF92CF9319
:105E8000DF93EC01688179818A819B8161157105BD
:105E90008105910521F464E279ED8BE597E02DE130
:105EA00033EF41E050E00E94C72E49015A019B01A7
:105EB000AC01A7EAB1E40E946E2E6B017C01ACEE4E
:105EC000B4EFA50194010E947C2EC60ED71EE81ED9
:105ED000F91EF7FE06C081E0C81AD108E10880E883
:105EE000F80AC882D982EA82FB82C701B6019F778D
:105EF000DF91CF91FF90EF90DF90CF90BF90AF9068
:105F00009F908F9008950E94372F089586E091E02A
:105F10000E94372F089560930601709307018093C4
:105F200008019093090108952F923F925F926F921A
:105F30007F928F929F92AF92BF92CF92DF92EF9219
:105F4000FF920F931F93CF93DF938B01EA016115AB
:105F5000710521F0DB018C9311969C93209739F009
:105F60009E01225031092332310508F0D8C07C014E
:105F70006701BFEFCB1ADB0A5601F7016080862D5F
:105F800090E00E94C630892B11F07601F1CFFDE23E
:105F90006F120AC0570182E0A80EB11CD7011196FA
:105FA0006C90772473940BC0BBE26B1207C057014F
:105FB000E2E0AE0EB11CD70111966C90712CCE01AF
:105FC0008F7E892B89F4B0E36B1237C0F501808195
:105FD0008F7D8835D1F46180F2E0AF0EB11C872D42
:105FE0008260782EC0E1D0E0CA30D10551F1C031D5
:105FF000D10521F0C830D10599F409C0CC24CA9448
:10600000DC2CEC2CAFE0FA2E22C0209769F7C8E018
:10601000D0E0CC24CA94DC2CEC2CFFE1FF2E17C07E
:106020006FEF7FEFCB019E01442737FD4095542F42
:106030000E94A52E69017A010AC02097A9F6CAE03C
:10604000D0E0E9E9CE2EDC2CEC2CE9E1FE2EF501C6
:1060500060E020E030E0A9014E01AA2497FCA09462
:10606000BA2C1F0170ED572E560CA9E0A51570F43F
:106070008FEB860D8A3118F499EC592E06C08FE902
:10608000860D8A3148F589EA582E560C852D90E008
:106090008C179D070CF56F3FD9F0C216D306E406A6
:1060A000F50698F0C501B4010E94812E9B01AC0158
:1060B000852D90E0A0E0B0E0280F391F4A1F5B1F3C
:1060C000281739074A075B0710F46FEF01C061E03A
:1060D0003196D1016C90C5CF0115110551F06623A1
:1060E00011F0319703C071FE04C03297D801ED93CF
:1060F000FC9370FE07C050954095309521953F4F19
:106100004F4F5F4F67FF10C082E290E090938D0683
:1061100080938C066FEF7FEF8FEF9FEF07C060E0FB
:1061200070E080E090E002C0B901CA01DF91CF9138
:106130001F910F91FF90EF90DF90CF90BF90AF90A5
:106140009F908F907F906F905F903F902F900895D9
:10615000FC0188279927E89421912032E9F329301E
:1061600010F02E30C8F32B3241F02D3239F4689400
:1061700004C00E94FA30820F911D219120532A30D1
:10618000C0F31EF4909581959F4F0895911150C0D2
:10619000803219F089508550D0F7089548EC53E0CB
:1061A0000E94D3300895FA01A191B081009719F4AB
:1061B0001097E1F0CD01DC01CD010D90002011F42C
:1061C000C00113C0FB012191222319F02015D9F73A
:1061D000F3CFFB012191201519F41E92119606C0F0
:1061E0002223C1F70D900020A1F7D001FA01A1935D
:1061F000B08308957AE0979F902D879F802D910D11
:1062000011240895F999FECF92BD81BDF89A99277E
:1062100080B50895262FF999FECF1FBA92BD81BD92
:1062200020BD0FB6F894FA9AF99A0FBE0196089518
:0A623000992788270895F894FFCFFE
:10623A0000008E06200001000000FF00020002009C
:10624A000200020002000200020002000200020034
:10625A00020002000200020002000280250000057E
:10626A00400AA1204EA50020244EA52C2330C0129E
:10627A0000001A400AA1204EA5001B1E27522C23FB
:10628A00308025000005400AA1204EA50020244E9A
:10629A00A52C2330004B000006400AD0009D49007F
:1062AA007B289D492C233000E1000005400A450166
:1062BA00D7DC03B81E0EBF00232E48E801008A402F
:1062CA000A6001555502AD1E20000023C80154582A
:1062DA002074696D656F75742100596573004E6F7E
:1062EA00002C00386368004E2F41002C205B005DB3
:1062FA002028002900486F70206368616E6E656C03
:10630A00200020402000456E746572696E67206126
:10631A0064617074697665206368616E6E656C206D
:10632A0073656C656374696F6E2C207069636B6941
:10633A006E673A007363616E6E6572206D6F646595
:10634A00004E4F5420454E41424C45440053656E21
:10635A0064696E672073657474696E677320746FFD
:10636A002052580A00526573657474696E67207307
:10637A00657474696E6773206F6E2052580A004103
:10638A00626F727465642065646974730A00696E69
:10639A0076616C69642073656C656374696F6E00FD
:1063AA000D0A496E76616C696420696E7075742095
:1063BA002D20646973636172646564210700536503
:1063CA007474696E677320736176656420746F20D4
:1063DA00454550524F4D0A005265766572746564A0
:1063EA002073657474696E67732066726F6D2045D9
:1063FA004550524F4D0A004C6F61646564206661D6
:10640A0063746F72792064656661756C74730A00CF
:10641A004B657920616E64206368616E6E656C738A
:10642A002072616E646F6D697A65640A004F7065E7
:10643A006E4C52536E67205458207374617274699B
:10644A006E672000206F6E20485720006D6F6475BC
:10645A006C65206C6F636B65643F00342B340038C5
:10646A0000382B340031320031322B3400313600FF
:10647A0050504D0052535349005344410053434C2A
:10648A0000525844005458440041494E004C424579
:10649A0045500053504B54524D00534255530053EC
:1064AA00554D44004C4C494E440000070B0C10114A
:1064BA001500B7012B032F033103350338033D03BE
:1064CA00B7014003440349034D03510355035903DC
:1064DA005D0363036A036F0374038D028D028D02E9
:1064EA008D02160A1322312900000000A72CAC2ABB
:0864FA004D2C7A2C5F2C9C2C28
:00000001FF
